:1000000009C021C020C01FC01EC01DC01CC01BC015
:100010001AC019C011241FBECFE9CDBF10E0A0E661
:10002000B0E0E2EEF1E002C005900D92A036B1071B
:10003000D9F710E0A0E6B0E001C01D92A636B107E6
:10004000E1F785D0CCC0DCCFB89AB99ABA9A8FEFD5
:1000500087BB089598E0C09880FDC09AC19A0000BF
:10006000C19886959150B9F7C29A0000C298089538
:10007000813481F49CEF9093600022E12093610031
:1000800031E13093620030936300209364009093D9
:10009000650026C0823489F49FEF9093600091E957
:1000A0009093610090936200909363009AEE909316
:1000B000640094E49093650024C0833489F49CE345
:1000C0009093600092E49093610021E82093620095
:1000D000209363009093640094E29093650023C0A2
:1000E000883479F48FEF809360008093610098E109
:1000F0009093620090936300809364008093650006
:1001000023C0803581F48FEF8093600089E0809375
:10011000610080936200809363008093640086E0B6
:100120008093650011C0893579F487E08093600081
:100130009FE09093610028E7209362002093630082
:10014000909364008093650080E690E00895CF93DB
:10015000DF93CDB7DEB7C450CDBF76DF81E492E444
:10016000A3E4B0E089839A83AB83BC836E010894D7
:10017000C11CD11C66247724F60101900020E9F708
:10018000CF0101978C199D0918161906ACF7560175
:100190004601880E991EF50181915F0169DFE82E05
:1001A000F92E8301F70181917F0154DF83EF91E004
:1001B0000197F1F700C000000F5F1F4F06301105D7
:1001C00089F780E047DFE1EEF4E03197F1F700C016
:1001D000000080E03FDFA814B90471F2DCCFF8948E
:0201E000FFCF4F
:00000001FF
